ARM Linker, 5.03 [Build 76] [MDK-ARM Standard]

==============================================================================

Section Cross References

    startup_stm32f407.o(RESET) refers to startup_stm32f407.o(STACK) for __initial_sp
    startup_stm32f407.o(RESET) refers to startup_stm32f407.o(.text) for Reset_Handler
    startup_stm32f407.o(RESET) refers to f_can_drive.o(.text) for CAN1_TX_IRQHandler
    startup_stm32f407.o(RESET) refers to f_inobus.o(.text) for TIM1_BRK_TIM9_IRQHandler
    startup_stm32f407.o(RESET) refers to f_uart.o(.text) for DMA2_Stream1_IRQHandler
    startup_stm32f407.o(.text) refers to main.o(.text) for SystemInit
    startup_stm32f407.o(.text) refers to entry.o(.ARM.Collect$$$$00000000) for __main
    system_stm32f4xx.o(.text) refers to system_stm32f4xx.o(.data) for SystemCoreClock
    stm32f4xx_can.o(.text) refers to stm32f4xx_rcc.o(.text) for RCC_APB1PeriphResetCmd
    stm32f4xx_gpio.o(.text) refers to stm32f4xx_rcc.o(.text) for RCC_AHB1PeriphResetCmd
    stm32f4xx_pwr.o(.text) refers to stm32f4xx_rcc.o(.text) for RCC_APB1PeriphResetCmd
    stm32f4xx_rcc.o(.text) refers to stm32f4xx_rcc.o(.data) for APBAHBPrescTable
    stm32f4xx_syscfg.o(.text) refers to stm32f4xx_rcc.o(.text) for RCC_APB2PeriphResetCmd
    stm32f4xx_tim.o(.text) refers to stm32f4xx_rcc.o(.text) for RCC_APB2PeriphResetCmd
    stm32f4xx_usart.o(.text) refers to stm32f4xx_rcc.o(.text) for RCC_APB2PeriphResetCmd
    stm32f4xx_wwdg.o(.text) refers to stm32f4xx_rcc.o(.text) for RCC_APB1PeriphResetCmd
    f_led.o(.text) refers to stm32f4xx_rcc.o(.text) for RCC_AHB1PeriphClockCmd
    f_led.o(.text) refers to stm32f4xx_gpio.o(.text) for GPIO_Init
    f_led.o(.text) refers to f_led.o(.constdata) for GPIO_CLK
    f_led.o(.text) refers to f_led.o(.data) for GPIO_PORT
    f_main.o(.text) refers to misc.o(.text) for NVIC_SetVectorTable
    f_main.o(.text) refers to stm32f4xx_rcc.o(.text) for RCC_APB1PeriphClockCmd
    f_main.o(.text) refers to stm32f4xx_tim.o(.text) for TIM_DeInit
    f_main.o(.text) refers to f_led.o(.text) for LED_Ctrl
    f_main.o(.text) refers to f_tech_comm_interface.o(.text) for SysInitDeal
    f_main.o(.text) refers to f_inobusif.o(.text) for C_InobusLoop
    f_main.o(.text) refers to f_user_main.o(.text) for userMainProc
    f_main.o(.text) refers to f_main.o(.bss) for LedPara
    f_main.o(.text) refers to f_tech_comm_interface.o(.data) for InoBusStatus
    f_main.o(.text) refers to f_main.o(.data) for SysInitStatusPre
    f_main.o(.text) refers to f_tech_comm_interface.o(.bss) for HcuParaCode
    f_main.o(.text) refers to f_user_main.o(.bss) for ParaCode
    f_tech_comm_interface.o(.text) refers to f_inobusif.o(.text) for C_SetPdLen
    f_tech_comm_interface.o(.text) refers to f_tech_comm_interface.o(.bss) for PdoDataBuff
    f_tech_comm_interface.o(.text) refers to f_tech_comm_interface.o(.data) for InoBusStatus
    f_wwdg.o(.text) refers to f_wwdg.o(.data) for FUNC_WWDG
    main.o(.text) refers to f_rcc.o(.text) for ClolkInit
    main.o(.text) refers to stm32f4xx_dbgmcu.o(.text) for DBGMCU_APB1PeriphConfig
    main.o(.text) refers to f_main.o(.text) for NVIC_Configuration
    main.o(.text) refers to f_inobusif.o(.text) for C_InobusLoop
    main.o(.text) refers to f_led.o(.text) for LED_IO_Init
    main.o(.text) refers to f_tech_comm_interface.o(.text) for SysInitVal
    main.o(.text) refers to f_wwdg.o(.text) for WatchDogInit
    main.o(.text) refers to f_user_main.o(.text) for userInitProc
    main.o(.text) refers to main.o(.data) for SysTimePre
    main.o(.text) refers to f_main.o(.bss) for SysTimeMonitor
    f_inobus.o(.text) refers to f_uart.o(.text) for Uart6DmaSend
    f_inobus.o(.text) refers to stm32f4xx_tim.o(.text) for TIM_GetITStatus
    f_inobus.o(.text) refers to stm32f4xx_rcc.o(.text) for RCC_APB1PeriphClockCmd
    f_inobus.o(.text) refers to f_inobusif.o(.text) for GetCardVesion
    f_inobus.o(.text) refers to stm32f4xx_usart.o(.text) for USART_SendData
    f_inobus.o(.text) refers to f_inobus.o(.bss) for UartSendBuf
    f_inobus.o(.text) refers to f_inobus.o(.data) for g_MsgValidFlag
    f_inobus.o(.text) refers to f_tech_comm_interface.o(.data) for PdoOffLineCnt
    f_inobus.o(.text) refers to memcpya.o(.text) for __aeabi_memcpy4
    f_inobus.o(.text) refers to misc.o(.text) for NVIC_Init
    f_inobusif.o(.text) refers to f_inobus.o(.text) for InobusMainLoop
    f_inobusif.o(.text) refers to f_tech_comm_interface.o(.text) for InobusAddrToFuncAddr
    f_inobusif.o(.text) refers to f_led.o(.text) for LED_Ctrl
    f_inobusif.o(.text) refers to f_tech_comm_interface.o(.bss) for PdoDataBuff
    f_inobusif.o(.text) refers to f_inobusif.o(.data) for OldStatus
    f_uart.o(.text) refers to stm32f4xx_dma.o(.text) for DMA_GetITStatus
    f_uart.o(.text) refers to stm32f4xx_usart.o(.text) for USART_DMACmd
    f_uart.o(.text) refers to f_inobus.o(.text) for UartTranOverCallback
    f_uart.o(.text) refers to stm32f4xx_rcc.o(.text) for RCC_AHB1PeriphClockCmd
    f_uart.o(.text) refers to misc.o(.text) for NVIC_Init
    f_uart.o(.text) refers to stm32f4xx_gpio.o(.text) for GPIO_PinAFConfig
    f_uart.o(.text) refers to f_uart.o(.bss) for RxDmaData
    f_uart.o(.text) refers to f_uart.o(.data) for pRecvData
    f_can_app.o(.text) refers to f_can_drive.o(.text) for InitRecMbox
    f_can_app.o(.text) refers to f_can_app.o(.data) for CANopenMode
    f_can_app.o(.text) refers to f_can_app.o(.bss) for TestBB
    f_can_app.o(.text) refers to f_can_app.o(.constdata) for CAN_ID_PDO_SEL_DEFAULT
    f_can_app.o(.text) refers to f_tech_comm_interface.o(.data) for SystemStatus
    f_can_app.o(.text) refers to f_user_main.o(.bss) for PdoData
    f_can_drive.o(.text) refers to memseta.o(.text) for __aeabi_memclr4
    f_can_drive.o(.text) refers to stm32f4xx_can.o(.text) for CAN_Transmit
    f_can_drive.o(.text) refers to memcpya.o(.text) for __aeabi_memcpy4
    f_can_drive.o(.text) refers to f_can_app.o(.text) for CANIntHook
    f_can_drive.o(.text) refers to stm32f4xx_gpio.o(.text) for GPIO_PinAFConfig
    f_can_drive.o(.text) refers to stm32f4xx_rcc.o(.text) for RCC_AHB1PeriphClockCmd
    f_can_drive.o(.text) refers to f_can_drive.o(.bss) for gCanTxBuf
    f_can_drive.o(.text) refers to f_can_drive.o(.data) for count
    f_can_drive.o(.text) refers to misc.o(.text) for NVIC_Init
    f_can_drive.o(.text) refers to f_can_drive.o(.constdata) for StCanBaud
    f_user_main.o(.text) refers to f_main.o(.text) for ModuleLed3GreenDispSet
    f_user_main.o(.text) refers to f_can_app.o(.text) for CanMainProcess
    f_user_main.o(.text) refers to f_can_app.o(.data) for CanTimeOutTicker
    f_user_main.o(.text) refers to f_user_main.o(.data) for TestLoad
    f_user_main.o(.text) refers to f_user_main.o(.bss) for PdoData
    entry.o(.ARM.Collect$$$$00000000) refers (Special) to entry10a.o(.ARM.Collect$$$$0000000D) for __rt_final_cpp
    entry.o(.ARM.Collect$$$$00000000) refers (Special) to entry11a.o(.ARM.Collect$$$$0000000F) for __rt_final_exit
    entry.o(.ARM.Collect$$$$00000000) refers (Special) to entry7b.o(.ARM.Collect$$$$00000008) for _main_clock
    entry.o(.ARM.Collect$$$$00000000) refers (Special) to entry8b.o(.ARM.Collect$$$$0000000A) for _main_cpp_init
    entry.o(.ARM.Collect$$$$00000000) refers (Special) to entry9a.o(.ARM.Collect$$$$0000000B) for _main_init
    entry.o(.ARM.Collect$$$$00000000) refers (Special) to entry5.o(.ARM.Collect$$$$00000004) for _main_scatterload
    entry.o(.ARM.Collect$$$$00000000) refers (Special) to entry2.o(.ARM.Collect$$$$00000001) for _main_stk
    entry2.o(.ARM.Collect$$$$00000001) refers to entry2.o(.ARM.Collect$$$$00002712) for __lit__00000000
    entry2.o(.ARM.Collect$$$$00002712) refers to startup_stm32f407.o(STACK) for __initial_sp
    entry2.o(__vectab_stack_and_reset_area) refers to startup_stm32f407.o(STACK) for __initial_sp
    entry2.o(__vectab_stack_and_reset_area) refers to entry.o(.ARM.Collect$$$$00000000) for __main
    entry5.o(.ARM.Collect$$$$00000004) refers to init.o(.text) for __scatterload
    entry9a.o(.ARM.Collect$$$$0000000B) refers to main.o(.text) for main
    entry9b.o(.ARM.Collect$$$$0000000C) refers to main.o(.text) for main
    init.o(.text) refers to entry5.o(.ARM.Collect$$$$00000004) for __main_after_scatterload


==============================================================================

Removing Unused input sections from the image.

    Removing startup_stm32f407.o(HEAP), (512 bytes).
    Removing system_stm32f4xx.o(.rev16_text), (4 bytes).
    Removing system_stm32f4xx.o(.revsh_text), (4 bytes).
    Removing system_stm32f4xx.o(.text), (192 bytes).
    Removing system_stm32f4xx.o(.data), (20 bytes).
    Removing misc.o(.rev16_text), (4 bytes).
    Removing misc.o(.revsh_text), (4 bytes).
    Removing stm32f4xx_can.o(.rev16_text), (4 bytes).
    Removing stm32f4xx_can.o(.revsh_text), (4 bytes).
    Removing stm32f4xx_dbgmcu.o(.rev16_text), (4 bytes).
    Removing stm32f4xx_dbgmcu.o(.revsh_text), (4 bytes).
    Removing stm32f4xx_dma.o(.rev16_text), (4 bytes).
    Removing stm32f4xx_dma.o(.revsh_text), (4 bytes).
    Removing stm32f4xx_exti.o(.rev16_text), (4 bytes).
    Removing stm32f4xx_exti.o(.revsh_text), (4 bytes).
    Removing stm32f4xx_exti.o(.text), (284 bytes).
    Removing stm32f4xx_flash.o(.rev16_text), (4 bytes).
    Removing stm32f4xx_flash.o(.revsh_text), (4 bytes).
    Removing stm32f4xx_flash.o(.text), (1224 bytes).
    Removing stm32f4xx_gpio.o(.rev16_text), (4 bytes).
    Removing stm32f4xx_gpio.o(.revsh_text), (4 bytes).
    Removing stm32f4xx_pwr.o(.rev16_text), (4 bytes).
    Removing stm32f4xx_pwr.o(.revsh_text), (4 bytes).
    Removing stm32f4xx_pwr.o(.text), (252 bytes).
    Removing stm32f4xx_rcc.o(.rev16_text), (4 bytes).
    Removing stm32f4xx_rcc.o(.revsh_text), (4 bytes).
    Removing stm32f4xx_syscfg.o(.rev16_text), (4 bytes).
    Removing stm32f4xx_syscfg.o(.revsh_text), (4 bytes).
    Removing stm32f4xx_syscfg.o(.text), (140 bytes).
    Removing stm32f4xx_tim.o(.rev16_text), (4 bytes).
    Removing stm32f4xx_tim.o(.revsh_text), (4 bytes).
    Removing stm32f4xx_usart.o(.rev16_text), (4 bytes).
    Removing stm32f4xx_usart.o(.revsh_text), (4 bytes).
    Removing stm32f4xx_wwdg.o(.rev16_text), (4 bytes).
    Removing stm32f4xx_wwdg.o(.revsh_text), (4 bytes).
    Removing stm32f4xx_wwdg.o(.text), (144 bytes).
    Removing f_led.o(.rev16_text), (4 bytes).
    Removing f_led.o(.revsh_text), (4 bytes).
    Removing f_main.o(.rev16_text), (4 bytes).
    Removing f_main.o(.revsh_text), (4 bytes).
    Removing f_rcc.o(.rev16_text), (4 bytes).
    Removing f_rcc.o(.revsh_text), (4 bytes).
    Removing f_tech_comm_interface.o(.rev16_text), (4 bytes).
    Removing f_tech_comm_interface.o(.revsh_text), (4 bytes).
    Removing main.o(.rev16_text), (4 bytes).
    Removing main.o(.revsh_text), (4 bytes).
    Removing f_inobus.o(.rev16_text), (4 bytes).
    Removing f_inobus.o(.revsh_text), (4 bytes).
    Removing f_inobusif.o(.rev16_text), (4 bytes).
    Removing f_inobusif.o(.revsh_text), (4 bytes).
    Removing f_uart.o(.rev16_text), (4 bytes).
    Removing f_uart.o(.revsh_text), (4 bytes).
    Removing f_can_app.o(.rev16_text), (4 bytes).
    Removing f_can_app.o(.revsh_text), (4 bytes).
    Removing f_can_drive.o(.rev16_text), (4 bytes).
    Removing f_can_drive.o(.revsh_text), (4 bytes).

56 unused section(s) (total 2960 bytes) removed from the image.

==============================================================================

Image Symbol Table

    Local Symbols

    Symbol Name                              Value     Ov Type        Size  Object(Section)

    ../clib/microlib/init/entry.s            0x00000000   Number         0  entry7b.o ABSOLUTE
    ../clib/microlib/init/entry.s            0x00000000   Number         0  entry10b.o ABSOLUTE
    ../clib/microlib/init/entry.s            0x00000000   Number         0  entry10a.o ABSOLUTE
    ../clib/microlib/init/entry.s            0x00000000   Number         0  entry9b.o ABSOLUTE
    ../clib/microlib/init/entry.s            0x00000000   Number         0  entry8b.o ABSOLUTE
    ../clib/microlib/init/entry.s            0x00000000   Number         0  entry2.o ABSOLUTE
    ../clib/microlib/init/entry.s            0x00000000   Number         0  entry9a.o ABSOLUTE
    ../clib/microlib/init/entry.s            0x00000000   Number         0  entry5.o ABSOLUTE
    ../clib/microlib/init/entry.s            0x00000000   Number         0  entry8a.o ABSOLUTE
    ../clib/microlib/init/entry.s            0x00000000   Number         0  entry7a.o ABSOLUTE
    ../clib/microlib/init/entry.s            0x00000000   Number         0  entry11a.o ABSOLUTE
    ../clib/microlib/init/entry.s            0x00000000   Number         0  entry.o ABSOLUTE
    ../clib/microlib/init/entry.s            0x00000000   Number         0  entry11b.o ABSOLUTE
    ../clib/microlib/string/memcpy.c         0x00000000   Number         0  memcpya.o ABSOLUTE
    ../clib/microlib/string/memcpy.c         0x00000000   Number         0  memcpyb.o ABSOLUTE
    ../clib/microlib/string/memset.c         0x00000000   Number         0  memseta.o ABSOLUTE
    ..\1_STM32F4xx_Lib\source\misc.c         0x00000000   Number         0  misc.o ABSOLUTE
    ..\1_STM32F4xx_Lib\source\stm32f4xx_can.c 0x00000000   Number         0  stm32f4xx_can.o ABSOLUTE
    ..\1_STM32F4xx_Lib\source\stm32f4xx_dbgmcu.c 0x00000000   Number         0  stm32f4xx_dbgmcu.o ABSOLUTE
    ..\1_STM32F4xx_Lib\source\stm32f4xx_dma.c 0x00000000   Number         0  stm32f4xx_dma.o ABSOLUTE
    ..\1_STM32F4xx_Lib\source\stm32f4xx_exti.c 0x00000000   Number         0  stm32f4xx_exti.o ABSOLUTE
    ..\1_STM32F4xx_Lib\source\stm32f4xx_flash.c 0x00000000   Number         0  stm32f4xx_flash.o ABSOLUTE
    ..\1_STM32F4xx_Lib\source\stm32f4xx_gpio.c 0x00000000   Number         0  stm32f4xx_gpio.o ABSOLUTE
    ..\1_STM32F4xx_Lib\source\stm32f4xx_pwr.c 0x00000000   Number         0  stm32f4xx_pwr.o ABSOLUTE
    ..\1_STM32F4xx_Lib\source\stm32f4xx_rcc.c 0x00000000   Number         0  stm32f4xx_rcc.o ABSOLUTE
    ..\1_STM32F4xx_Lib\source\stm32f4xx_syscfg.c 0x00000000   Number         0  stm32f4xx_syscfg.o ABSOLUTE
    ..\1_STM32F4xx_Lib\source\stm32f4xx_tim.c 0x00000000   Number         0  stm32f4xx_tim.o ABSOLUTE
    ..\1_STM32F4xx_Lib\source\stm32f4xx_usart.c 0x00000000   Number         0  stm32f4xx_usart.o ABSOLUTE
    ..\1_STM32F4xx_Lib\source\stm32f4xx_wwdg.c 0x00000000   Number         0  stm32f4xx_wwdg.o ABSOLUTE
    ..\2_CMSIS\source\startup_stm32f407.s    0x00000000   Number         0  startup_stm32f407.o ABSOLUTE
    ..\2_CMSIS\source\system_stm32f4xx.c     0x00000000   Number         0  system_stm32f4xx.o ABSOLUTE
    ..\3_User\1_Public\source\f_Led.c        0x00000000   Number         0  f_led.o ABSOLUTE
    ..\3_User\1_Public\source\f_main.c       0x00000000   Number         0  f_main.o ABSOLUTE
    ..\3_User\1_Public\source\f_rcc.c        0x00000000   Number         0  f_rcc.o ABSOLUTE
    ..\3_User\1_Public\source\f_tech_comm_interface.c 0x00000000   Number         0  f_tech_comm_interface.o ABSOLUTE
    ..\3_User\1_Public\source\f_wwdg.c       0x00000000   Number         0  f_wwdg.o ABSOLUTE
    ..\3_User\1_Public\source\main.c         0x00000000   Number         0  main.o ABSOLUTE
    ..\3_User\2_Inobus\source\F_InobusIf.c   0x00000000   Number         0  f_inobusif.o ABSOLUTE
    ..\3_User\2_Inobus\source\f_inobus.c     0x00000000   Number         0  f_inobus.o ABSOLUTE
    ..\3_User\2_Inobus\source\f_uart.c       0x00000000   Number         0  f_uart.o ABSOLUTE
    ..\3_User\3_can\source\f_CAN_app.c       0x00000000   Number         0  f_can_app.o ABSOLUTE
    ..\3_User\3_can\source\f_CAN_drive.c     0x00000000   Number         0  f_can_drive.o ABSOLUTE
    ..\3_User\99_User_Defined\source\f_user_main.c 0x00000000   Number         0  f_user_main.o ABSOLUTE
    ..\\1_STM32F4xx_Lib\\source\\misc.c      0x00000000   Number         0  misc.o ABSOLUTE
    ..\\1_STM32F4xx_Lib\\source\\stm32f4xx_can.c 0x00000000   Number         0  stm32f4xx_can.o ABSOLUTE
    ..\\1_STM32F4xx_Lib\\source\\stm32f4xx_dbgmcu.c 0x00000000   Number         0  stm32f4xx_dbgmcu.o ABSOLUTE
    ..\\1_STM32F4xx_Lib\\source\\stm32f4xx_dma.c 0x00000000   Number         0  stm32f4xx_dma.o ABSOLUTE
    ..\\1_STM32F4xx_Lib\\source\\stm32f4xx_exti.c 0x00000000   Number         0  stm32f4xx_exti.o ABSOLUTE
    ..\\1_STM32F4xx_Lib\\source\\stm32f4xx_flash.c 0x00000000   Number         0  stm32f4xx_flash.o ABSOLUTE
    ..\\1_STM32F4xx_Lib\\source\\stm32f4xx_gpio.c 0x00000000   Number         0  stm32f4xx_gpio.o ABSOLUTE
    ..\\1_STM32F4xx_Lib\\source\\stm32f4xx_pwr.c 0x00000000   Number         0  stm32f4xx_pwr.o ABSOLUTE
    ..\\1_STM32F4xx_Lib\\source\\stm32f4xx_rcc.c 0x00000000   Number         0  stm32f4xx_rcc.o ABSOLUTE
    ..\\1_STM32F4xx_Lib\\source\\stm32f4xx_syscfg.c 0x00000000   Number         0  stm32f4xx_syscfg.o ABSOLUTE
    ..\\1_STM32F4xx_Lib\\source\\stm32f4xx_tim.c 0x00000000   Number         0  stm32f4xx_tim.o ABSOLUTE
    ..\\1_STM32F4xx_Lib\\source\\stm32f4xx_usart.c 0x00000000   Number         0  stm32f4xx_usart.o ABSOLUTE
    ..\\1_STM32F4xx_Lib\\source\\stm32f4xx_wwdg.c 0x00000000   Number         0  stm32f4xx_wwdg.o ABSOLUTE
    ..\\2_CMSIS\\source\\system_stm32f4xx.c  0x00000000   Number         0  system_stm32f4xx.o ABSOLUTE
    ..\\3_User\\1_Public\\source\\f_Led.c    0x00000000   Number         0  f_led.o ABSOLUTE
    ..\\3_User\\1_Public\\source\\f_main.c   0x00000000   Number         0  f_main.o ABSOLUTE
    ..\\3_User\\1_Public\\source\\f_rcc.c    0x00000000   Number         0  f_rcc.o ABSOLUTE
    ..\\3_User\\1_Public\\source\\f_tech_comm_interface.c 0x00000000   Number         0  f_tech_comm_interface.o ABSOLUTE
    ..\\3_User\\1_Public\\source\\main.c     0x00000000   Number         0  main.o ABSOLUTE
    ..\\3_User\\2_Inobus\\source\\F_InobusIf.c 0x00000000   Number         0  f_inobusif.o ABSOLUTE
    ..\\3_User\\2_Inobus\\source\\f_inobus.c 0x00000000   Number         0  f_inobus.o ABSOLUTE
    ..\\3_User\\2_Inobus\\source\\f_uart.c   0x00000000   Number         0  f_uart.o ABSOLUTE
    ..\\3_User\\3_can\\source\\f_CAN_app.c   0x00000000   Number         0  f_can_app.o ABSOLUTE
    ..\\3_User\\3_can\\source\\f_CAN_drive.c 0x00000000   Number         0  f_can_drive.o ABSOLUTE
    dc.s                                     0x00000000   Number         0  dc.o ABSOLUTE
    handlers.s                               0x00000000   Number         0  handlers.o ABSOLUTE
    init.s                                   0x00000000   Number         0  init.o ABSOLUTE
    RESET                                    0x08000000   Section      392  startup_stm32f407.o(RESET)
    .ARM.Collect$$$$00000000                 0x08000188   Section        0  entry.o(.ARM.Collect$$$$00000000)
    .ARM.Collect$$$$00000001                 0x08000188   Section        4  entry2.o(.ARM.Collect$$$$00000001)
    .ARM.Collect$$$$00000004                 0x0800018c   Section        4  entry5.o(.ARM.Collect$$$$00000004)
    .ARM.Collect$$$$00000008                 0x08000190   Section        0  entry7b.o(.ARM.Collect$$$$00000008)
    .ARM.Collect$$$$0000000A                 0x08000190   Section        0  entry8b.o(.ARM.Collect$$$$0000000A)
    .ARM.Collect$$$$0000000B                 0x08000190   Section        8  entry9a.o(.ARM.Collect$$$$0000000B)
    .ARM.Collect$$$$0000000D                 0x08000198   Section        0  entry10a.o(.ARM.Collect$$$$0000000D)
    .ARM.Collect$$$$0000000F                 0x08000198   Section        0  entry11a.o(.ARM.Collect$$$$0000000F)
    .ARM.Collect$$$$00002712                 0x08000198   Section        4  entry2.o(.ARM.Collect$$$$00002712)
    __lit__00000000                          0x08000198   Data           4  entry2.o(.ARM.Collect$$$$00002712)
    .text                                    0x0800019c   Section       36  startup_stm32f407.o(.text)
    $v0                                      0x0800019c   Number         0  startup_stm32f407.o(.text)
    .text                                    0x080001c0   Section        0  misc.o(.text)
    .text                                    0x080002a4   Section        0  stm32f4xx_can.o(.text)
    CheckITStatus                            0x08000aa7   Thumb Code    16  stm32f4xx_can.o(.text)
    .text                                    0x08000c90   Section        0  stm32f4xx_dbgmcu.o(.text)
    .text                                    0x08000cf4   Section        0  stm32f4xx_dma.o(.text)
    .text                                    0x08001098   Section        0  stm32f4xx_gpio.o(.text)
    .text                                    0x080012f4   Section        0  stm32f4xx_rcc.o(.text)
    .text                                    0x0800187c   Section        0  stm32f4xx_tim.o(.text)
    TI4_Config                               0x0800201b   Thumb Code    80  stm32f4xx_tim.o(.text)
    TI3_Config                               0x0800207d   Thumb Code    72  stm32f4xx_tim.o(.text)
    TI2_Config                               0x080020df   Thumb Code    90  stm32f4xx_tim.o(.text)
    TI1_Config                               0x0800214b   Thumb Code    58  stm32f4xx_tim.o(.text)
    .text                                    0x08002520   Section        0  stm32f4xx_usart.o(.text)
    .text                                    0x0800293c   Section        0  f_led.o(.text)
    .text                                    0x08002a5c   Section        0  f_main.o(.text)
    ModuleLedCtrl                            0x08002ab9   Thumb Code   220  f_main.o(.text)
    ModuleLedDeal                            0x08002b95   Thumb Code    40  f_main.o(.text)
    UpdateLedStatus                          0x08002bd5   Thumb Code   156  f_main.o(.text)
    UpdateDataToUserApp                      0x08002c71   Thumb Code   182  f_main.o(.text)
    .text                                    0x08002ea4   Section        0  f_rcc.o(.text)
    SetSysClock                              0x08002ea5   Thumb Code   190  f_rcc.o(.text)
    .text                                    0x080030c4   Section        0  f_tech_comm_interface.o(.text)
    .text                                    0x0800339c   Section        0  f_wwdg.o(.text)
    .text                                    0x08003424   Section        0  main.o(.text)
    .text                                    0x080034e0   Section        0  f_inobus.o(.text)
    CrcCaculate                              0x080034e1   Thumb Code    68  f_inobus.o(.text)
    Ino_SendNormalData                       0x08003525   Thumb Code   296  f_inobus.o(.text)
    TIM3_Configuration                       0x0800366f   Thumb Code    58  f_inobus.o(.text)
    InobusInitDsp                            0x080036a9   Thumb Code    12  f_inobus.o(.text)
    Ino_SendHandshake                        0x080036b7   Thumb Code    68  f_inobus.o(.text)
    GetSyncPeriod                            0x080036fb   Thumb Code    12  f_inobus.o(.text)
    Ino_MsgWatchDog                          0x08003755   Thumb Code   114  f_inobus.o(.text)
    InoProcessNormal                         0x080037c7   Thumb Code   246  f_inobus.o(.text)
    Ino_RxDataProcess                        0x080038bd   Thumb Code   298  f_inobus.o(.text)
    .text                                    0x08003bb8   Section        0  f_inobusif.o(.text)
    .text                                    0x08003d8c   Section        0  f_uart.o(.text)
    .text                                    0x08004090   Section        0  f_can_app.o(.text)
    CanFilterConfigDeal                      0x08004091   Thumb Code   122  f_can_app.o(.text)
    .text                                    0x080042c0   Section        0  f_can_drive.o(.text)
    CanDataSendDemo                          0x080043a5   Thumb Code   110  f_can_drive.o(.text)
    NVIC_EnableIRQ                           0x08004a87   Thumb Code    24  f_can_drive.o(.text)
    .text                                    0x08004ab0   Section        0  f_user_main.o(.text)
    .text                                    0x08004b24   Section        0  memcpya.o(.text)
    .text                                    0x08004b48   Section        0  memseta.o(.text)
    .text                                    0x08004b6c   Section       36  init.o(.text)
    i.__scatterload_copy                     0x08004b90   Section       14  handlers.o(i.__scatterload_copy)
    i.__scatterload_null                     0x08004b9e   Section        2  handlers.o(i.__scatterload_null)
    i.__scatterload_zeroinit                 0x08004ba0   Section       14  handlers.o(i.__scatterload_zeroinit)
    .constdata                               0x08004bb0   Section       56  f_led.o(.constdata)
    .constdata                               0x08004be8   Section       32  f_can_app.o(.constdata)
    .constdata                               0x08004c08   Section       42  f_can_drive.o(.constdata)
    .data                                    0x20000000   Section       16  stm32f4xx_rcc.o(.data)
    APBAHBPrescTable                         0x20000000   Data          16  stm32f4xx_rcc.o(.data)
    .data                                    0x20000010   Section       36  f_led.o(.data)
    .data                                    0x20000034   Section        8  f_main.o(.data)
    SysInitStatusPre                         0x20000034   Data           2  f_main.o(.data)
    .data                                    0x2000003c   Section       20  f_tech_comm_interface.o(.data)
    TimeOutCnt                               0x20000046   Data           2  f_tech_comm_interface.o(.data)
    TickerOk                                 0x20000048   Data           2  f_tech_comm_interface.o(.data)
    TickerWait                               0x2000004a   Data           2  f_tech_comm_interface.o(.data)
    flag                                     0x2000004c   Data           2  f_tech_comm_interface.o(.data)
    TimeCnt                                  0x2000004e   Data           2  f_tech_comm_interface.o(.data)
    .data                                    0x20000050   Section        4  f_wwdg.o(.data)
    .data                                    0x20000054   Section        2  main.o(.data)
    SysTimePre                               0x20000054   Data           2  main.o(.data)
    .data                                    0x20000058   Section       32  f_inobus.o(.data)
    InoInitFlag                              0x2000005a   Data           2  f_inobus.o(.data)
    HandshakeCnt                             0x2000005c   Data           2  f_inobus.o(.data)
    DeviceStatus                             0x2000005e   Data           2  f_inobus.o(.data)
    CardStatus                               0x20000060   Data           2  f_inobus.o(.data)
    g_InoLedStatus                           0x20000062   Data           1  f_inobus.o(.data)
    g_MsgValidFlag                           0x20000063   Data           1  f_inobus.o(.data)
    g_PdPoint                                0x20000064   Data           2  f_inobus.o(.data)
    g_HeartbeatCnt                           0x20000066   Data           2  f_inobus.o(.data)
    .data                                    0x20000078   Section       11  f_inobusif.o(.data)
    OldStatus                                0x20000078   Data           2  f_inobusif.o(.data)
    LedOnCnt                                 0x2000007a   Data           2  f_inobusif.o(.data)
    LedOffCnt                                0x2000007c   Data           2  f_inobusif.o(.data)
    HostLedOnTime                            0x2000007e   Data           2  f_inobusif.o(.data)
    HostLedOffTime                           0x20000080   Data           2  f_inobusif.o(.data)
    HostActLed                               0x20000082   Data           1  f_inobusif.o(.data)
    .data                                    0x20000084   Section        8  f_uart.o(.data)
    .data                                    0x2000008c   Section       16  f_can_app.o(.data)
    CanInitalStep                            0x20000096   Data           2  f_can_app.o(.data)
    .data                                    0x2000009c   Section        4  f_can_drive.o(.data)
    con                                      0x2000009c   Data           2  f_can_drive.o(.data)
    count                                    0x2000009e   Data           2  f_can_drive.o(.data)
    .data                                    0x200000a0   Section        4  f_user_main.o(.data)
    .bss                                     0x200000a4   Section      118  f_main.o(.bss)
    .bss                                     0x2000011a   Section       94  f_tech_comm_interface.o(.bss)
    .bss                                     0x20000178   Section     1816  f_inobus.o(.bss)
    SendMsgBuf                               0x20000178   Data         778  f_inobus.o(.bss)
    .bss                                     0x20000890   Section      512  f_uart.o(.bss)
    .bss                                     0x20000a90   Section       52  f_can_app.o(.bss)
    .bss                                     0x20000ac4   Section      352  f_can_drive.o(.bss)
    .bss                                     0x20000c24   Section       94  f_user_main.o(.bss)
    STACK                                    0x20000c88   Section     4096  startup_stm32f407.o(STACK)

    Global Symbols

    Symbol Name                              Value     Ov Type        Size  Object(Section)

    BuildAttributes$$THM_ISAv4$E$P$D$K$B$S$7EM$VFPi3$EXTD16$VFPS$VFMA$PE$A:L22UL41UL21$X:L11$S22US41US21$IEEE1$IW$USESV6$~STKCKD$USESV7$~SHL$OSPACE$EBA8$MICROLIB$REQ8$PRES8$EABIv2 0x00000000   Number         0  anon$$obj.o ABSOLUTE
    __ARM_use_no_argv                        0x00000000   Number         0  main.o ABSOLUTE
    __cpp_initialize__aeabi_                  - Undefined Weak Reference
    __cxa_finalize                            - Undefined Weak Reference
    __decompress                              - Undefined Weak Reference
    _clock_init                               - Undefined Weak Reference
    _microlib_exit                            - Undefined Weak Reference
    __Vectors_Size                           0x00000188   Number         0  startup_stm32f407.o ABSOLUTE
    __Vectors                                0x08000000   Data           4  startup_stm32f407.o(RESET)
    __Vectors_End                            0x08000188   Data           0  startup_stm32f407.o(RESET)
    __main                                   0x08000189   Thumb Code     0  entry.o(.ARM.Collect$$$$00000000)
    _main_stk                                0x08000189   Thumb Code     0  entry2.o(.ARM.Collect$$$$00000001)
    _main_scatterload                        0x0800018d   Thumb Code     0  entry5.o(.ARM.Collect$$$$00000004)
    __main_after_scatterload                 0x08000191   Thumb Code     0  entry5.o(.ARM.Collect$$$$00000004)
    _main_clock                              0x08000191   Thumb Code     0  entry7b.o(.ARM.Collect$$$$00000008)
    _main_cpp_init                           0x08000191   Thumb Code     0  entry8b.o(.ARM.Collect$$$$0000000A)
    _main_init                               0x08000191   Thumb Code     0  entry9a.o(.ARM.Collect$$$$0000000B)
    __rt_final_cpp                           0x08000199   Thumb Code     0  entry10a.o(.ARM.Collect$$$$0000000D)
    __rt_final_exit                          0x08000199   Thumb Code     0  entry11a.o(.ARM.Collect$$$$0000000F)
    Reset_Handler                            0x0800019d   Thumb Code     8  startup_stm32f407.o(.text)
    NMI_Handler                              0x080001a5   Thumb Code     2  startup_stm32f407.o(.text)
    HardFault_Handler                        0x080001a7   Thumb Code     2  startup_stm32f407.o(.text)
    MemManage_Handler                        0x080001a9   Thumb Code     2  startup_stm32f407.o(.text)
    BusFault_Handler                         0x080001ab   Thumb Code     2  startup_stm32f407.o(.text)
    UsageFault_Handler                       0x080001ad   Thumb Code     2  startup_stm32f407.o(.text)
    SVC_Handler                              0x080001af   Thumb Code     2  startup_stm32f407.o(.text)
    DebugMon_Handler                         0x080001b1   Thumb Code     2  startup_stm32f407.o(.text)
    PendSV_Handler                           0x080001b3   Thumb Code     2  startup_stm32f407.o(.text)
    SysTick_Handler                          0x080001b5   Thumb Code     2  startup_stm32f407.o(.text)
    ADC_IRQHandler                           0x080001b7   Thumb Code     0  startup_stm32f407.o(.text)
    CAN1_SCE_IRQHandler                      0x080001b7   Thumb Code     0  startup_stm32f407.o(.text)
    CAN2_RX0_IRQHandler                      0x080001b7   Thumb Code     0  startup_stm32f407.o(.text)
    CAN2_RX1_IRQHandler                      0x080001b7   Thumb Code     0  startup_stm32f407.o(.text)
    CAN2_SCE_IRQHandler                      0x080001b7   Thumb Code     0  startup_stm32f407.o(.text)
    CAN2_TX_IRQHandler                       0x080001b7   Thumb Code     0  startup_stm32f407.o(.text)
    CRYP_IRQHandler                          0x080001b7   Thumb Code     0  startup_stm32f407.o(.text)
    DCMI_IRQHandler                          0x080001b7   Thumb Code     0  startup_stm32f407.o(.text)
    DMA1_Stream0_IRQHandler                  0x080001b7   Thumb Code     0  startup_stm32f407.o(.text)
    DMA1_Stream1_IRQHandler                  0x080001b7   Thumb Code     0  startup_stm32f407.o(.text)
    DMA1_Stream2_IRQHandler                  0x080001b7   Thumb Code     0  startup_stm32f407.o(.text)
    DMA1_Stream3_IRQHandler                  0x080001b7   Thumb Code     0  startup_stm32f407.o(.text)
    DMA1_Stream4_IRQHandler                  0x080001b7   Thumb Code     0  startup_stm32f407.o(.text)
    DMA1_Stream5_IRQHandler                  0x080001b7   Thumb Code     0  startup_stm32f407.o(.text)
    DMA1_Stream6_IRQHandler                  0x080001b7   Thumb Code     0  startup_stm32f407.o(.text)
    DMA1_Stream7_IRQHandler                  0x080001b7   Thumb Code     0  startup_stm32f407.o(.text)
    DMA2_Stream0_IRQHandler                  0x080001b7   Thumb Code     0  startup_stm32f407.o(.text)
    DMA2_Stream2_IRQHandler                  0x080001b7   Thumb Code     0  startup_stm32f407.o(.text)
    DMA2_Stream3_IRQHandler                  0x080001b7   Thumb Code     0  startup_stm32f407.o(.text)
    DMA2_Stream4_IRQHandler                  0x080001b7   Thumb Code     0  startup_stm32f407.o(.text)
    DMA2_Stream5_IRQHandler                  0x080001b7   Thumb Code     0  startup_stm32f407.o(.text)
    DMA2_Stream7_IRQHandler                  0x080001b7   Thumb Code     0  startup_stm32f407.o(.text)
    ETH_IRQHandler                           0x080001b7   Thumb Code     0  startup_stm32f407.o(.text)
    ETH_WKUP_IRQHandler                      0x080001b7   Thumb Code     0  startup_stm32f407.o(.text)
    EXTI0_IRQHandler                         0x080001b7   Thumb Code     0  startup_stm32f407.o(.text)
    EXTI15_10_IRQHandler                     0x080001b7   Thumb Code     0  startup_stm32f407.o(.text)
    EXTI1_IRQHandler                         0x080001b7   Thumb Code     0  startup_stm32f407.o(.text)
    EXTI2_IRQHandler                         0x080001b7   Thumb Code     0  startup_stm32f407.o(.text)
    EXTI3_IRQHandler                         0x080001b7   Thumb Code     0  startup_stm32f407.o(.text)
    EXTI4_IRQHandler                         0x080001b7   Thumb Code     0  startup_stm32f407.o(.text)
    EXTI9_5_IRQHandler                       0x080001b7   Thumb Code     0  startup_stm32f407.o(.text)
    FLASH_IRQHandler                         0x080001b7   Thumb Code     0  startup_stm32f407.o(.text)
    FPU_IRQHandler                           0x080001b7   Thumb Code     0  startup_stm32f407.o(.text)
    FSMC_IRQHandler                          0x080001b7   Thumb Code     0  startup_stm32f407.o(.text)
    HASH_RNG_IRQHandler                      0x080001b7   Thumb Code     0  startup_stm32f407.o(.text)
    I2C1_ER_IRQHandler                       0x080001b7   Thumb Code     0  startup_stm32f407.o(.text)
    I2C1_EV_IRQHandler                       0x080001b7   Thumb Code     0  startup_stm32f407.o(.text)
    I2C2_ER_IRQHandler                       0x080001b7   Thumb Code     0  startup_stm32f407.o(.text)
    I2C2_EV_IRQHandler                       0x080001b7   Thumb Code     0  startup_stm32f407.o(.text)
    I2C3_ER_IRQHandler                       0x080001b7   Thumb Code     0  startup_stm32f407.o(.text)
    I2C3_EV_IRQHandler                       0x080001b7   Thumb Code     0  startup_stm32f407.o(.text)
    OTG_FS_IRQHandler                        0x080001b7   Thumb Code     0  startup_stm32f407.o(.text)
    OTG_FS_WKUP_IRQHandler                   0x080001b7   Thumb Code     0  startup_stm32f407.o(.text)
    OTG_HS_EP1_IN_IRQHandler                 0x080001b7   Thumb Code     0  startup_stm32f407.o(.text)
    OTG_HS_EP1_OUT_IRQHandler                0x080001b7   Thumb Code     0  startup_stm32f407.o(.text)
    OTG_HS_IRQHandler                        0x080001b7   Thumb Code     0  startup_stm32f407.o(.text)
    OTG_HS_WKUP_IRQHandler                   0x080001b7   Thumb Code     0  startup_stm32f407.o(.text)
    PVD_IRQHandler                           0x080001b7   Thumb Code     0  startup_stm32f407.o(.text)
    RCC_IRQHandler                           0x080001b7   Thumb Code     0  startup_stm32f407.o(.text)
    RTC_Alarm_IRQHandler                     0x080001b7   Thumb Code     0  startup_stm32f407.o(.text)
    RTC_WKUP_IRQHandler                      0x080001b7   Thumb Code     0  startup_stm32f407.o(.text)
    SDIO_IRQHandler                          0x080001b7   Thumb Code     0  startup_stm32f407.o(.text)
    SPI1_IRQHandler                          0x080001b7   Thumb Code     0  startup_stm32f407.o(.text)
    SPI2_IRQHandler                          0x080001b7   Thumb Code     0  startup_stm32f407.o(.text)
    SPI3_IRQHandler                          0x080001b7   Thumb Code     0  startup_stm32f407.o(.text)
    TAMP_STAMP_IRQHandler                    0x080001b7   Thumb Code     0  startup_stm32f407.o(.text)
    TIM1_CC_IRQHandler                       0x080001b7   Thumb Code     0  startup_stm32f407.o(.text)
    TIM1_TRG_COM_TIM11_IRQHandler            0x080001b7   Thumb Code     0  startup_stm32f407.o(.text)
    TIM1_UP_TIM10_IRQHandler                 0x080001b7   Thumb Code     0  startup_stm32f407.o(.text)
    TIM2_IRQHandler                          0x080001b7   Thumb Code     0  startup_stm32f407.o(.text)
    TIM3_IRQHandler                          0x080001b7   Thumb Code     0  startup_stm32f407.o(.text)
    TIM4_IRQHandler                          0x080001b7   Thumb Code     0  startup_stm32f407.o(.text)
    TIM5_IRQHandler                          0x080001b7   Thumb Code     0  startup_stm32f407.o(.text)
    TIM6_DAC_IRQHandler                      0x080001b7   Thumb Code     0  startup_stm32f407.o(.text)
    TIM7_IRQHandler                          0x080001b7   Thumb Code     0  startup_stm32f407.o(.text)
    TIM8_BRK_TIM12_IRQHandler                0x080001b7   Thumb Code     0  startup_stm32f407.o(.text)
    TIM8_CC_IRQHandler                       0x080001b7   Thumb Code     0  startup_stm32f407.o(.text)
    TIM8_TRG_COM_TIM14_IRQHandler            0x080001b7   Thumb Code     0  startup_stm32f407.o(.text)
    TIM8_UP_TIM13_IRQHandler                 0x080001b7   Thumb Code     0  startup_stm32f407.o(.text)
    UART4_IRQHandler                         0x080001b7   Thumb Code     0  startup_stm32f407.o(.text)
    UART5_IRQHandler                         0x080001b7   Thumb Code     0  startup_stm32f407.o(.text)
    USART1_IRQHandler                        0x080001b7   Thumb Code     0  startup_stm32f407.o(.text)
    USART2_IRQHandler                        0x080001b7   Thumb Code     0  startup_stm32f407.o(.text)
    USART3_IRQHandler                        0x080001b7   Thumb Code     0  startup_stm32f407.o(.text)
    WWDG_IRQHandler                          0x080001b7   Thumb Code     0  startup_stm32f407.o(.text)
    NVIC_PriorityGroupConfig                 0x080001c1   Thumb Code    10  misc.o(.text)
    NVIC_Init                                0x080001cb   Thumb Code   108  misc.o(.text)
    NVIC_SetVectorTable                      0x08000237   Thumb Code    14  misc.o(.text)
    NVIC_SystemLPConfig                      0x08000245   Thumb Code    34  misc.o(.text)
    SysTick_CLKSourceConfig                  0x08000267   Thumb Code    40  misc.o(.text)
    CAN_DeInit                               0x080002a5   Thumb Code    50  stm32f4xx_can.o(.text)
    CAN_Init                                 0x080002d7   Thumb Code   276  stm32f4xx_can.o(.text)
    CAN_FilterInit                           0x080003eb   Thumb Code   258  stm32f4xx_can.o(.text)
    CAN_StructInit                           0x080004ed   Thumb Code    32  stm32f4xx_can.o(.text)
    CAN_SlaveStartBank                       0x0800050d   Thumb Code    48  stm32f4xx_can.o(.text)
    CAN_DBGFreeze                            0x0800053d   Thumb Code    22  stm32f4xx_can.o(.text)
    CAN_TTComModeCmd                         0x08000553   Thumb Code   118  stm32f4xx_can.o(.text)
    CAN_Transmit                             0x080005c9   Thumb Code   304  stm32f4xx_can.o(.text)
    CAN_TransmitStatus                       0x080006f9   Thumb Code   138  stm32f4xx_can.o(.text)
    CAN_CancelTransmit                       0x08000783   Thumb Code    48  stm32f4xx_can.o(.text)
    CAN_Receive                              0x080007b3   Thumb Code   240  stm32f4xx_can.o(.text)
    CAN_FIFORelease                          0x080008a3   Thumb Code    22  stm32f4xx_can.o(.text)
    CAN_MessagePending                       0x080008b9   Thumb Code    30  stm32f4xx_can.o(.text)
    CAN_OperatingModeRequest                 0x080008d7   Thumb Code   162  stm32f4xx_can.o(.text)
    CAN_Sleep                                0x08000979   Thumb Code    30  stm32f4xx_can.o(.text)
    CAN_WakeUp                               0x08000997   Thumb Code    48  stm32f4xx_can.o(.text)
    CAN_GetLastErrorCode                     0x080009c7   Thumb Code    12  stm32f4xx_can.o(.text)
    CAN_GetReceiveErrorCounter               0x080009d3   Thumb Code    10  stm32f4xx_can.o(.text)
    CAN_GetLSBTransmitErrorCounter           0x080009dd   Thumb Code    12  stm32f4xx_can.o(.text)
    CAN_ITConfig                             0x080009e9   Thumb Code    18  stm32f4xx_can.o(.text)
    CAN_GetFlagStatus                        0x080009fb   Thumb Code   120  stm32f4xx_can.o(.text)
    CAN_ClearFlag                            0x08000a73   Thumb Code    52  stm32f4xx_can.o(.text)
    CAN_GetITStatus                          0x08000ab7   Thumb Code   308  stm32f4xx_can.o(.text)
    CAN_ClearITPendingBit                    0x08000beb   Thumb Code   162  stm32f4xx_can.o(.text)
    DBGMCU_GetREVID                          0x08000c91   Thumb Code     8  stm32f4xx_dbgmcu.o(.text)
    DBGMCU_GetDEVID                          0x08000c99   Thumb Code    10  stm32f4xx_dbgmcu.o(.text)
    DBGMCU_Config                            0x08000ca3   Thumb Code    26  stm32f4xx_dbgmcu.o(.text)
    DBGMCU_APB1PeriphConfig                  0x08000cbd   Thumb Code    26  stm32f4xx_dbgmcu.o(.text)
    DBGMCU_APB2PeriphConfig                  0x08000cd7   Thumb Code    26  stm32f4xx_dbgmcu.o(.text)
    DMA_DeInit                               0x08000cf5   Thumb Code   324  stm32f4xx_dma.o(.text)
    DMA_Init                                 0x08000e39   Thumb Code    82  stm32f4xx_dma.o(.text)
    DMA_StructInit                           0x08000e8b   Thumb Code    34  stm32f4xx_dma.o(.text)
    DMA_Cmd                                  0x08000ead   Thumb Code    22  stm32f4xx_dma.o(.text)
    DMA_PeriphIncOffsetSizeConfig            0x08000ec3   Thumb Code    22  stm32f4xx_dma.o(.text)
    DMA_FlowControllerConfig                 0x08000ed9   Thumb Code    22  stm32f4xx_dma.o(.text)
    DMA_SetCurrDataCounter                   0x08000eef   Thumb Code     4  stm32f4xx_dma.o(.text)
    DMA_GetCurrDataCounter                   0x08000ef3   Thumb Code     8  stm32f4xx_dma.o(.text)
    DMA_DoubleBufferModeConfig               0x08000efb   Thumb Code    24  stm32f4xx_dma.o(.text)
    DMA_DoubleBufferModeCmd                  0x08000f13   Thumb Code    22  stm32f4xx_dma.o(.text)
    DMA_MemoryTargetConfig                   0x08000f29   Thumb Code    10  stm32f4xx_dma.o(.text)
    DMA_GetCurrentMemoryTarget               0x08000f33   Thumb Code    20  stm32f4xx_dma.o(.text)
    DMA_GetCmdStatus                         0x08000f47   Thumb Code    20  stm32f4xx_dma.o(.text)
    DMA_GetFIFOStatus                        0x08000f5b   Thumb Code    12  stm32f4xx_dma.o(.text)
    DMA_GetFlagStatus                        0x08000f67   Thumb Code    54  stm32f4xx_dma.o(.text)
    DMA_ClearFlag                            0x08000f9d   Thumb Code    40  stm32f4xx_dma.o(.text)
    DMA_ITConfig                             0x08000fc5   Thumb Code    58  stm32f4xx_dma.o(.text)
    DMA_GetITStatus                          0x08000fff   Thumb Code    82  stm32f4xx_dma.o(.text)
    DMA_ClearITPendingBit                    0x08001051   Thumb Code    40  stm32f4xx_dma.o(.text)
    GPIO_DeInit                              0x08001099   Thumb Code   220  stm32f4xx_gpio.o(.text)
    GPIO_Init                                0x08001175   Thumb Code   144  stm32f4xx_gpio.o(.text)
    GPIO_StructInit                          0x08001205   Thumb Code    18  stm32f4xx_gpio.o(.text)
    GPIO_PinLockConfig                       0x08001217   Thumb Code    34  stm32f4xx_gpio.o(.text)
    GPIO_ReadInputDataBit                    0x08001239   Thumb Code    18  stm32f4xx_gpio.o(.text)
    GPIO_ReadInputData                       0x0800124b   Thumb Code     8  stm32f4xx_gpio.o(.text)
    GPIO_ReadOutputDataBit                   0x08001253   Thumb Code    18  stm32f4xx_gpio.o(.text)
    GPIO_ReadOutputData                      0x08001265   Thumb Code     8  stm32f4xx_gpio.o(.text)
    GPIO_SetBits                             0x0800126d   Thumb Code     4  stm32f4xx_gpio.o(.text)
    GPIO_ResetBits                           0x08001271   Thumb Code     4  stm32f4xx_gpio.o(.text)
    GPIO_WriteBit                            0x08001275   Thumb Code    10  stm32f4xx_gpio.o(.text)
    GPIO_Write                               0x0800127f   Thumb Code     4  stm32f4xx_gpio.o(.text)
    GPIO_ToggleBits                          0x08001283   Thumb Code     8  stm32f4xx_gpio.o(.text)
    GPIO_PinAFConfig                         0x0800128b   Thumb Code    70  stm32f4xx_gpio.o(.text)
    RCC_DeInit                               0x080012f5   Thumb Code    60  stm32f4xx_rcc.o(.text)
    RCC_HSEConfig                            0x08001331   Thumb Code    14  stm32f4xx_rcc.o(.text)
    RCC_GetFlagStatus                        0x0800133f   Thumb Code    60  stm32f4xx_rcc.o(.text)
    RCC_WaitForHSEStartUp                    0x0800137b   Thumb Code    56  stm32f4xx_rcc.o(.text)
    RCC_AdjustHSICalibrationValue            0x080013b3   Thumb Code    20  stm32f4xx_rcc.o(.text)
    RCC_HSICmd                               0x080013c7   Thumb Code     6  stm32f4xx_rcc.o(.text)
    RCC_LSEConfig                            0x080013cd   Thumb Code    46  stm32f4xx_rcc.o(.text)
    RCC_LSICmd                               0x080013fb   Thumb Code     6  stm32f4xx_rcc.o(.text)
    RCC_PLLConfig                            0x08001401   Thumb Code    32  stm32f4xx_rcc.o(.text)
    RCC_PLLCmd                               0x08001421   Thumb Code     6  stm32f4xx_rcc.o(.text)
    RCC_PLLI2SConfig                         0x08001427   Thumb Code    14  stm32f4xx_rcc.o(.text)
    RCC_PLLI2SCmd                            0x08001435   Thumb Code     6  stm32f4xx_rcc.o(.text)
    RCC_ClockSecuritySystemCmd               0x0800143b   Thumb Code     6  stm32f4xx_rcc.o(.text)
    RCC_MCO1Config                           0x08001441   Thumb Code    28  stm32f4xx_rcc.o(.text)
    RCC_MCO2Config                           0x0800145d   Thumb Code    28  stm32f4xx_rcc.o(.text)
    RCC_SYSCLKConfig                         0x08001479   Thumb Code    20  stm32f4xx_rcc.o(.text)
    RCC_GetSYSCLKSource                      0x0800148d   Thumb Code    12  stm32f4xx_rcc.o(.text)
    RCC_HCLKConfig                           0x08001499   Thumb Code    20  stm32f4xx_rcc.o(.text)
    RCC_PCLK1Config                          0x080014ad   Thumb Code    20  stm32f4xx_rcc.o(.text)
    RCC_PCLK2Config                          0x080014c1   Thumb Code    22  stm32f4xx_rcc.o(.text)
    RCC_GetClocksFreq                        0x080014d7   Thumb Code   222  stm32f4xx_rcc.o(.text)
    RCC_RTCCLKConfig                         0x080015b5   Thumb Code    54  stm32f4xx_rcc.o(.text)
    RCC_RTCCLKCmd                            0x080015eb   Thumb Code     8  stm32f4xx_rcc.o(.text)
    RCC_BackupResetCmd                       0x080015f3   Thumb Code     8  stm32f4xx_rcc.o(.text)
    RCC_I2SCLKConfig                         0x080015fb   Thumb Code     6  stm32f4xx_rcc.o(.text)
    RCC_AHB1PeriphClockCmd                   0x08001601   Thumb Code    34  stm32f4xx_rcc.o(.text)
    RCC_AHB2PeriphClockCmd                   0x08001623   Thumb Code    34  stm32f4xx_rcc.o(.text)
    RCC_AHB3PeriphClockCmd                   0x08001645   Thumb Code    34  stm32f4xx_rcc.o(.text)
    RCC_APB1PeriphClockCmd                   0x08001667   Thumb Code    34  stm32f4xx_rcc.o(.text)
    RCC_APB2PeriphClockCmd                   0x08001689   Thumb Code    34  stm32f4xx_rcc.o(.text)
    RCC_AHB1PeriphResetCmd                   0x080016ab   Thumb Code    34  stm32f4xx_rcc.o(.text)
    RCC_AHB2PeriphResetCmd                   0x080016cd   Thumb Code    72  stm32f4xx_rcc.o(.text)
    RCC_AHB3PeriphResetCmd                   0x08001715   Thumb Code    34  stm32f4xx_rcc.o(.text)
    RCC_APB1PeriphResetCmd                   0x08001737   Thumb Code    34  stm32f4xx_rcc.o(.text)
    RCC_APB2PeriphResetCmd                   0x08001759   Thumb Code    34  stm32f4xx_rcc.o(.text)
    RCC_AHB1PeriphClockLPModeCmd             0x0800177b   Thumb Code    34  stm32f4xx_rcc.o(.text)
    RCC_AHB2PeriphClockLPModeCmd             0x0800179d   Thumb Code    34  stm32f4xx_rcc.o(.text)
    RCC_AHB3PeriphClockLPModeCmd             0x080017bf   Thumb Code    34  stm32f4xx_rcc.o(.text)
    RCC_APB1PeriphClockLPModeCmd             0x080017e1   Thumb Code    34  stm32f4xx_rcc.o(.text)
    RCC_APB2PeriphClockLPModeCmd             0x08001803   Thumb Code    34  stm32f4xx_rcc.o(.text)
    RCC_ITConfig                             0x08001825   Thumb Code    34  stm32f4xx_rcc.o(.text)
    RCC_ClearFlag                            0x08001847   Thumb Code    18  stm32f4xx_rcc.o(.text)
    RCC_GetITStatus                          0x08001859   Thumb Code    22  stm32f4xx_rcc.o(.text)
    RCC_ClearITPendingBit                    0x0800186f   Thumb Code     8  stm32f4xx_rcc.o(.text)
    TIM_DeInit                               0x0800187d   Thumb Code   346  stm32f4xx_tim.o(.text)
    TIM_TimeBaseInit                         0x080019d7   Thumb Code   104  stm32f4xx_tim.o(.text)
    TIM_TimeBaseStructInit                   0x08001a3f   Thumb Code    18  stm32f4xx_tim.o(.text)
    TIM_PrescalerConfig                      0x08001a51   Thumb Code     6  stm32f4xx_tim.o(.text)
    TIM_CounterModeConfig                    0x08001a57   Thumb Code    18  stm32f4xx_tim.o(.text)
    TIM_SetCounter                           0x08001a69   Thumb Code     4  stm32f4xx_tim.o(.text)
    TIM_SetAutoreload                        0x08001a6d   Thumb Code     4  stm32f4xx_tim.o(.text)
    TIM_GetCounter                           0x08001a71   Thumb Code     6  stm32f4xx_tim.o(.text)
    TIM_GetPrescaler                         0x08001a77   Thumb Code     6  stm32f4xx_tim.o(.text)
    TIM_UpdateDisableConfig                  0x08001a7d   Thumb Code    24  stm32f4xx_tim.o(.text)
    TIM_UpdateRequestConfig                  0x08001a95   Thumb Code    24  stm32f4xx_tim.o(.text)
    TIM_ARRPreloadConfig                     0x08001aad   Thumb Code    24  stm32f4xx_tim.o(.text)
    TIM_SelectOnePulseMode                   0x08001ac5   Thumb Code    18  stm32f4xx_tim.o(.text)
    TIM_SetClockDivision                     0x08001ad7   Thumb Code    18  stm32f4xx_tim.o(.text)
    TIM_Cmd                                  0x08001ae9   Thumb Code    24  stm32f4xx_tim.o(.text)
    TIM_OC1Init                              0x08001b01   Thumb Code   114  stm32f4xx_tim.o(.text)
    TIM_OC2Init                              0x08001b73   Thumb Code   154  stm32f4xx_tim.o(.text)
    TIM_OC3Init                              0x08001c0d   Thumb Code   204  stm32f4xx_tim.o(.text)
    TIM_OC4Init                              0x08001cd9   Thumb Code   112  stm32f4xx_tim.o(.text)
    TIM_OCStructInit                         0x08001d49   Thumb Code    20  stm32f4xx_tim.o(.text)
    TIM_SelectOCxM                           0x08001d5d   Thumb Code    86  stm32f4xx_tim.o(.text)
    TIM_SetCompare1                          0x08001db3   Thumb Code     4  stm32f4xx_tim.o(.text)
    TIM_SetCompare2                          0x08001db7   Thumb Code     4  stm32f4xx_tim.o(.text)
    TIM_SetCompare3                          0x08001dbb   Thumb Code     4  stm32f4xx_tim.o(.text)
    TIM_SetCompare4                          0x08001dbf   Thumb Code     4  stm32f4xx_tim.o(.text)
    TIM_ForcedOC1Config                      0x08001dc3   Thumb Code    18  stm32f4xx_tim.o(.text)
    TIM_ForcedOC2Config                      0x08001dd5   Thumb Code    26  stm32f4xx_tim.o(.text)
    TIM_ForcedOC3Config                      0x08001def   Thumb Code    18  stm32f4xx_tim.o(.text)
    TIM_ForcedOC4Config                      0x08001e01   Thumb Code    26  stm32f4xx_tim.o(.text)
    TIM_OC1PreloadConfig                     0x08001e1b   Thumb Code    18  stm32f4xx_tim.o(.text)
    TIM_OC2PreloadConfig                     0x08001e2d   Thumb Code    26  stm32f4xx_tim.o(.text)
    TIM_OC3PreloadConfig                     0x08001e47   Thumb Code    18  stm32f4xx_tim.o(.text)
    TIM_OC4PreloadConfig                     0x08001e59   Thumb Code    26  stm32f4xx_tim.o(.text)
    TIM_OC1FastConfig                        0x08001e73   Thumb Code    18  stm32f4xx_tim.o(.text)
    TIM_OC2FastConfig                        0x08001e85   Thumb Code    26  stm32f4xx_tim.o(.text)
    TIM_OC3FastConfig                        0x08001e9f   Thumb Code    18  stm32f4xx_tim.o(.text)
    TIM_OC4FastConfig                        0x08001eb1   Thumb Code    26  stm32f4xx_tim.o(.text)
    TIM_ClearOC1Ref                          0x08001ecb   Thumb Code    18  stm32f4xx_tim.o(.text)
    TIM_ClearOC2Ref                          0x08001edd   Thumb Code    24  stm32f4xx_tim.o(.text)
    TIM_ClearOC3Ref                          0x08001ef5   Thumb Code    18  stm32f4xx_tim.o(.text)
    TIM_ClearOC4Ref                          0x08001f07   Thumb Code    24  stm32f4xx_tim.o(.text)
    TIM_OC1PolarityConfig                    0x08001f1f   Thumb Code    18  stm32f4xx_tim.o(.text)
    TIM_OC1NPolarityConfig                   0x08001f31   Thumb Code    18  stm32f4xx_tim.o(.text)
    TIM_OC2PolarityConfig                    0x08001f43   Thumb Code    26  stm32f4xx_tim.o(.text)
    TIM_OC2NPolarityConfig                   0x08001f5d   Thumb Code    26  stm32f4xx_tim.o(.text)
    TIM_OC3PolarityConfig                    0x08001f77   Thumb Code    26  stm32f4xx_tim.o(.text)
    TIM_OC3NPolarityConfig                   0x08001f91   Thumb Code    26  stm32f4xx_tim.o(.text)
    TIM_OC4PolarityConfig                    0x08001fab   Thumb Code    26  stm32f4xx_tim.o(.text)
    TIM_CCxCmd                               0x08001fc5   Thumb Code    30  stm32f4xx_tim.o(.text)
    TIM_CCxNCmd                              0x08001fe3   Thumb Code    30  stm32f4xx_tim.o(.text)
    TIM_SetIC4Prescaler                      0x08002001   Thumb Code    26  stm32f4xx_tim.o(.text)
    TIM_SetIC3Prescaler                      0x0800206b   Thumb Code    18  stm32f4xx_tim.o(.text)
    TIM_SetIC2Prescaler                      0x080020c5   Thumb Code    26  stm32f4xx_tim.o(.text)
    TIM_SetIC1Prescaler                      0x08002139   Thumb Code    18  stm32f4xx_tim.o(.text)
    TIM_ICInit                               0x08002185   Thumb Code   110  stm32f4xx_tim.o(.text)
    TIM_ICStructInit                         0x080021f3   Thumb Code    18  stm32f4xx_tim.o(.text)
    TIM_PWMIConfig                           0x08002205   Thumb Code   124  stm32f4xx_tim.o(.text)
    TIM_GetCapture1                          0x08002281   Thumb Code     6  stm32f4xx_tim.o(.text)
    TIM_GetCapture2                          0x08002287   Thumb Code     6  stm32f4xx_tim.o(.text)
    TIM_GetCapture3                          0x0800228d   Thumb Code     6  stm32f4xx_tim.o(.text)
    TIM_GetCapture4                          0x08002293   Thumb Code     6  stm32f4xx_tim.o(.text)
    TIM_BDTRConfig                           0x08002299   Thumb Code    32  stm32f4xx_tim.o(.text)
    TIM_BDTRStructInit                       0x080022b9   Thumb Code    18  stm32f4xx_tim.o(.text)
    TIM_CtrlPWMOutputs                       0x080022cb   Thumb Code    30  stm32f4xx_tim.o(.text)
    TIM_SelectCOM                            0x080022e9   Thumb Code    24  stm32f4xx_tim.o(.text)
    TIM_CCPreloadControl                     0x08002301   Thumb Code    24  stm32f4xx_tim.o(.text)
    TIM_ITConfig                             0x08002319   Thumb Code    18  stm32f4xx_tim.o(.text)
    TIM_GenerateEvent                        0x0800232b   Thumb Code     4  stm32f4xx_tim.o(.text)
    TIM_GetFlagStatus                        0x0800232f   Thumb Code    18  stm32f4xx_tim.o(.text)
    TIM_ClearFlag                            0x08002341   Thumb Code     6  stm32f4xx_tim.o(.text)
    TIM_GetITStatus                          0x08002347   Thumb Code    34  stm32f4xx_tim.o(.text)
    TIM_ClearITPendingBit                    0x08002369   Thumb Code     6  stm32f4xx_tim.o(.text)
    TIM_DMAConfig                            0x0800236f   Thumb Code    10  stm32f4xx_tim.o(.text)
    TIM_DMACmd                               0x08002379   Thumb Code    18  stm32f4xx_tim.o(.text)
    TIM_SelectCCDMA                          0x0800238b   Thumb Code    24  stm32f4xx_tim.o(.text)
    TIM_InternalClockConfig                  0x080023a3   Thumb Code    12  stm32f4xx_tim.o(.text)
    TIM_SelectInputTrigger                   0x080023af   Thumb Code    18  stm32f4xx_tim.o(.text)
    TIM_ITRxExternalClockConfig              0x080023c1   Thumb Code    24  stm32f4xx_tim.o(.text)
    TIM_TIxExternalClockConfig               0x080023d9   Thumb Code    62  stm32f4xx_tim.o(.text)
    TIM_ETRConfig                            0x08002417   Thumb Code    28  stm32f4xx_tim.o(.text)
    TIM_ETRClockMode1Config                  0x08002433   Thumb Code    54  stm32f4xx_tim.o(.text)
    TIM_ETRClockMode2Config                  0x08002469   Thumb Code    32  stm32f4xx_tim.o(.text)
    TIM_SelectOutputTrigger                  0x08002489   Thumb Code    18  stm32f4xx_tim.o(.text)
    TIM_SelectSlaveMode                      0x0800249b   Thumb Code    18  stm32f4xx_tim.o(.text)
    TIM_SelectMasterSlaveMode                0x080024ad   Thumb Code    18  stm32f4xx_tim.o(.text)
    TIM_EncoderInterfaceConfig               0x080024bf   Thumb Code    66  stm32f4xx_tim.o(.text)
    TIM_SelectHallSensor                     0x08002501   Thumb Code    24  stm32f4xx_tim.o(.text)
    TIM_RemapConfig                          0x08002519   Thumb Code     6  stm32f4xx_tim.o(.text)
    USART_DeInit                             0x08002521   Thumb Code   156  stm32f4xx_usart.o(.text)
    USART_Init                               0x080025bd   Thumb Code   204  stm32f4xx_usart.o(.text)
    USART_StructInit                         0x08002689   Thumb Code    24  stm32f4xx_usart.o(.text)
    USART_ClockInit                          0x080026a1   Thumb Code    32  stm32f4xx_usart.o(.text)
    USART_ClockStructInit                    0x080026c1   Thumb Code    12  stm32f4xx_usart.o(.text)
    USART_Cmd                                0x080026cd   Thumb Code    24  stm32f4xx_usart.o(.text)
    USART_SetPrescaler                       0x080026e5   Thumb Code    16  stm32f4xx_usart.o(.text)
    USART_OverSampling8Cmd                   0x080026f5   Thumb Code    22  stm32f4xx_usart.o(.text)
    USART_OneBitMethodCmd                    0x0800270b   Thumb Code    24  stm32f4xx_usart.o(.text)
    USART_SendData                           0x08002723   Thumb Code     8  stm32f4xx_usart.o(.text)
    USART_ReceiveData                        0x0800272b   Thumb Code    10  stm32f4xx_usart.o(.text)
    USART_SetAddress                         0x08002735   Thumb Code    18  stm32f4xx_usart.o(.text)
    USART_ReceiverWakeUpCmd                  0x08002747   Thumb Code    24  stm32f4xx_usart.o(.text)
    USART_WakeUpConfig                       0x0800275f   Thumb Code    18  stm32f4xx_usart.o(.text)
    USART_LINBreakDetectLengthConfig         0x08002771   Thumb Code    18  stm32f4xx_usart.o(.text)
    USART_LINCmd                             0x08002783   Thumb Code    24  stm32f4xx_usart.o(.text)
    USART_SendBreak                          0x0800279b   Thumb Code    10  stm32f4xx_usart.o(.text)
    USART_HalfDuplexCmd                      0x080027a5   Thumb Code    24  stm32f4xx_usart.o(.text)
    USART_SetGuardTime                       0x080027bd   Thumb Code    16  stm32f4xx_usart.o(.text)
    USART_SmartCardCmd                       0x080027cd   Thumb Code    24  stm32f4xx_usart.o(.text)
    USART_SmartCardNACKCmd                   0x080027e5   Thumb Code    24  stm32f4xx_usart.o(.text)
    USART_IrDAConfig                         0x080027fd   Thumb Code    18  stm32f4xx_usart.o(.text)
    USART_IrDACmd                            0x0800280f   Thumb Code    24  stm32f4xx_usart.o(.text)
    USART_DMACmd                             0x08002827   Thumb Code    18  stm32f4xx_usart.o(.text)
    USART_ITConfig                           0x08002839   Thumb Code    74  stm32f4xx_usart.o(.text)
    USART_GetFlagStatus                      0x08002883   Thumb Code    26  stm32f4xx_usart.o(.text)
    USART_ClearFlag                          0x0800289d   Thumb Code    18  stm32f4xx_usart.o(.text)
    USART_GetITStatus                        0x080028af   Thumb Code   110  stm32f4xx_usart.o(.text)
    USART_ClearITPendingBit                  0x0800291d   Thumb Code    30  stm32f4xx_usart.o(.text)
    STM_LEDInit                              0x0800293d   Thumb Code    62  f_led.o(.text)
    STM_LEDOn                                0x0800297b   Thumb Code    16  f_led.o(.text)
    STM_LEDOff                               0x0800298b   Thumb Code    16  f_led.o(.text)
    STM_LEDToggle                            0x0800299b   Thumb Code    26  f_led.o(.text)
    LED_Ctrl                                 0x080029b5   Thumb Code    26  f_led.o(.text)
    LED_IO_Init                              0x080029cf   Thumb Code   130  f_led.o(.text)
    NVIC_Configuration                       0x08002a5d   Thumb Code    22  f_main.o(.text)
    TIM4_Configuration                       0x08002a73   Thumb Code    58  f_main.o(.text)
    GetSysTime_1MHzClk                       0x08002aad   Thumb Code    12  f_main.o(.text)
    ModuleLed2GreenDispSet                   0x08002bbd   Thumb Code     8  f_main.o(.text)
    ModuleLed2OrangeDispSet                  0x08002bc5   Thumb Code     8  f_main.o(.text)
    ModuleLed2RedDispSet                     0x08002bcd   Thumb Code     8  f_main.o(.text)
    ManufacMainLoop                          0x08002d27   Thumb Code    44  f_main.o(.text)
    UsersMainLoop                            0x08002d53   Thumb Code    24  f_main.o(.text)
    SysMonitorDeal                           0x08002d6b   Thumb Code   132  f_main.o(.text)
    GetSysLoadRealTime                       0x08002def   Thumb Code     6  f_main.o(.text)
    GetSysLoadMax                            0x08002df5   Thumb Code     6  f_main.o(.text)
    InitModuleLedPara                        0x08002dfb   Thumb Code    64  f_main.o(.text)
    ModuleLed1RedDispSet                     0x08002e3b   Thumb Code     8  f_main.o(.text)
    ModuleLed1GreenDispSet                   0x08002e43   Thumb Code     8  f_main.o(.text)
    ModuleLed1OrangeDispSet                  0x08002e4b   Thumb Code     8  f_main.o(.text)
    ModuleLed3RedDispSet                     0x08002e53   Thumb Code    54  f_main.o(.text)
    ModuleLed3GreenDispSet                   0x08002e89   Thumb Code    12  f_main.o(.text)
    ModuleLed3OrangeDispSet                  0x08002e95   Thumb Code    12  f_main.o(.text)
    ClolkInit                                0x08002f63   Thumb Code    74  f_rcc.o(.text)
    PeripheralClockConfig                    0x08002fad   Thumb Code   256  f_rcc.o(.text)
    SysInitVal                               0x080030c5   Thumb Code    52  f_tech_comm_interface.o(.text)
    FuncCodeRead                             0x080030f9   Thumb Code    38  f_tech_comm_interface.o(.text)
    SysInitDeal                              0x0800311f   Thumb Code   258  f_tech_comm_interface.o(.text)
    HcuParaReadPeriod                        0x08003221   Thumb Code    94  f_tech_comm_interface.o(.text)
    InobusAddrToFuncAddr                     0x0800327f   Thumb Code    38  f_tech_comm_interface.o(.text)
    C_Read_Func_Response                     0x080032a5   Thumb Code   200  f_tech_comm_interface.o(.text)
    WatchDogInit                             0x0800339d   Thumb Code    92  f_wwdg.o(.text)
    ServiceDog                               0x080033f9   Thumb Code    20  f_wwdg.o(.text)
    DisableWDog                              0x0800340d   Thumb Code    18  f_wwdg.o(.text)
    SystemInit                               0x08003425   Thumb Code    44  main.o(.text)
    main                                     0x08003451   Thumb Code   132  main.o(.text)
    TIM1_BRK_TIM9_IRQHandler                 0x0800364d   Thumb Code    34  f_inobus.o(.text)
    Set_PdMappingAddr                        0x080036b5   Thumb Code     2  f_inobus.o(.text)
    Ino_SendSync                             0x08003707   Thumb Code    78  f_inobus.o(.text)
    InobusMainLoop                           0x080039e7   Thumb Code   138  f_inobus.o(.text)
    MsgSendDeal                              0x08003a71   Thumb Code   102  f_inobus.o(.text)
    InoSetPdLen                              0x08003ad7   Thumb Code    40  f_inobus.o(.text)
    Ino_GetDevStatus                         0x08003aff   Thumb Code     6  f_inobus.o(.text)
    Ino_SetCardStatus                        0x08003b05   Thumb Code     6  f_inobus.o(.text)
    Ino_GetBusOnline                         0x08003b0b   Thumb Code    14  f_inobus.o(.text)
    TIM9_Configuration                       0x08003b19   Thumb Code    86  f_inobus.o(.text)
    UartTranOverCallback                     0x08003b6f   Thumb Code     8  f_inobus.o(.text)
    UartRecvRdyCallback                      0x08003b77   Thumb Code    12  f_inobus.o(.text)
    C_InobusLoop                             0x08003bb9   Thumb Code     8  f_inobusif.o(.text)
    C_Read_FunCode                           0x08003bc1   Thumb Code    82  f_inobusif.o(.text)
    Ino_GetPdAddr                            0x08003c13   Thumb Code    16  f_inobusif.o(.text)
    C_SetPdLen                               0x08003c23   Thumb Code    16  f_inobusif.o(.text)
    C_DeviceAppState                         0x08003c33   Thumb Code     8  f_inobusif.o(.text)
    C_GetInobusOnline                        0x08003c3b   Thumb Code     8  f_inobusif.o(.text)
    CommStateSet                             0x08003c43   Thumb Code    12  f_inobusif.o(.text)
    C_AppSyncRecv                            0x08003c4f   Thumb Code     8  f_inobusif.o(.text)
    InoMsgRspCallbackFunc                    0x08003c57   Thumb Code   104  f_inobusif.o(.text)
    GetCardType                              0x08003cbf   Thumb Code     4  f_inobusif.o(.text)
    GetCardVesion                            0x08003cc3   Thumb Code     4  f_inobusif.o(.text)
    Host_Led_Proc                            0x08003cc7   Thumb Code   168  f_inobusif.o(.text)
    DMA2_Stream1_IRQHandler                  0x08003d8d   Thumb Code    32  f_uart.o(.text)
    DMA2_Stream6_IRQHandler                  0x08003dad   Thumb Code    58  f_uart.o(.text)
    USART6_IRQHandler                        0x08003de7   Thumb Code   170  f_uart.o(.text)
    Uart6InitDma                             0x08003e91   Thumb Code   204  f_uart.o(.text)
    Uart_GPIO_Init                           0x08003f5d   Thumb Code    54  f_uart.o(.text)
    Uart_Init                                0x08003f93   Thumb Code   136  f_uart.o(.text)
    Uart6DmaSend                             0x0800401b   Thumb Code    78  f_uart.o(.text)
    InitCanConfig                            0x0800410b   Thumb Code    44  f_can_app.o(.text)
    CanMainProcess                           0x08004137   Thumb Code   204  f_can_app.o(.text)
    CANRxdDataDeal                           0x08004203   Thumb Code   132  f_can_app.o(.text)
    CANIntHook                               0x08004287   Thumb Code    16  f_can_app.o(.text)
    eCanDataTran                             0x080042c1   Thumb Code   228  f_can_drive.o(.text)
    CAN1_RX0_IRQHandler                      0x08004413   Thumb Code   264  f_can_drive.o(.text)
    CAN1_RX1_IRQHandler                      0x0800451b   Thumb Code   264  f_can_drive.o(.text)
    CAN1_TX_IRQHandler                       0x08004623   Thumb Code   104  f_can_drive.o(.text)
    InitCANIO                                0x0800468b   Thumb Code    58  f_can_drive.o(.text)
    InitCanDrive                             0x080046c5   Thumb Code   802  f_can_drive.o(.text)
    InitRecMbox                              0x080049e7   Thumb Code   160  f_can_drive.o(.text)
    userInitProc                             0x08004ab1   Thumb Code     2  f_user_main.o(.text)
    UserLedCtrlTest                          0x08004ab3   Thumb Code    54  f_user_main.o(.text)
    userMainProc                             0x08004ae9   Thumb Code    42  f_user_main.o(.text)
    __aeabi_memcpy                           0x08004b25   Thumb Code    36  memcpya.o(.text)
    __aeabi_memcpy4                          0x08004b25   Thumb Code     0  memcpya.o(.text)
    __aeabi_memcpy8                          0x08004b25   Thumb Code     0  memcpya.o(.text)
    __aeabi_memset                           0x08004b49   Thumb Code    14  memseta.o(.text)
    __aeabi_memset4                          0x08004b49   Thumb Code     0  memseta.o(.text)
    __aeabi_memset8                          0x08004b49   Thumb Code     0  memseta.o(.text)
    __aeabi_memclr                           0x08004b57   Thumb Code     4  memseta.o(.text)
    __aeabi_memclr4                          0x08004b57   Thumb Code     0  memseta.o(.text)
    __aeabi_memclr8                          0x08004b57   Thumb Code     0  memseta.o(.text)
    _memset$wrapper                          0x08004b5b   Thumb Code    18  memseta.o(.text)
    __scatterload                            0x08004b6d   Thumb Code    28  init.o(.text)
    __scatterload_rt2                        0x08004b6d   Thumb Code     0  init.o(.text)
    __scatterload_copy                       0x08004b91   Thumb Code    14  handlers.o(i.__scatterload_copy)
    __scatterload_null                       0x08004b9f   Thumb Code     2  handlers.o(i.__scatterload_null)
    __scatterload_zeroinit                   0x08004ba1   Thumb Code    14  handlers.o(i.__scatterload_zeroinit)
    GPIO_PIN                                 0x08004bb0   Data          18  f_led.o(.constdata)
    GPIO_CLK                                 0x08004bc4   Data          36  f_led.o(.constdata)
    CAN_ID_PDO_SEL_DEFAULT                   0x08004be8   Data          32  f_can_app.o(.constdata)
    StCanBaud                                0x08004c08   Data          42  f_can_drive.o(.constdata)
    Region$$Table$$Base                      0x08004c34   Number         0  anon$$obj.o(Region$$Table)
    Region$$Table$$Limit                     0x08004c54   Number         0  anon$$obj.o(Region$$Table)
    GPIO_PORT                                0x20000010   Data          36  f_led.o(.data)
    testX1                                   0x20000036   Data           6  f_main.o(.data)
    InoBusStatus                             0x2000003c   Data           2  f_tech_comm_interface.o(.data)
    ModuleIdOkFlag                           0x2000003e   Data           2  f_tech_comm_interface.o(.data)
    SysInitStatus                            0x20000040   Data           1  f_tech_comm_interface.o(.data)
    PdoOffLineCnt                            0x20000042   Data           2  f_tech_comm_interface.o(.data)
    SystemStatus                             0x20000044   Data           2  f_tech_comm_interface.o(.data)
    FUNC_WWDG                                0x20000050   Data           4  f_wwdg.o(.data)
    InoOnlineFlag                            0x20000058   Data           1  f_inobus.o(.data)
    PdWrBuf                                  0x20000068   Data           8  f_inobus.o(.data)
    PdRdBuf                                  0x20000070   Data           8  f_inobus.o(.data)
    TxDmaInitData                            0x20000084   Data           1  f_uart.o(.data)
    pRecvData                                0x20000088   Data           4  f_uart.o(.data)
    CanParam                                 0x2000008c   Data           6  f_can_app.o(.data)
    CanTimeOutTicker                         0x20000092   Data           2  f_can_app.o(.data)
    CANopenMode                              0x20000094   Data           1  f_can_app.o(.data)
    CanState                                 0x20000098   Data           4  f_can_app.o(.data)
    TestLoad                                 0x200000a0   Data           2  f_user_main.o(.data)
    TestLoadMax                              0x200000a2   Data           2  f_user_main.o(.data)
    SysTimeMonitor                           0x200000a4   Data          28  f_main.o(.bss)
    LedPara                                  0x200000c0   Data          90  f_main.o(.bss)
    HcuParaCode                              0x2000011a   Data          30  f_tech_comm_interface.o(.bss)
    PdoDataBuff                              0x20000138   Data          64  f_tech_comm_interface.o(.bss)
    UartSendBuf                              0x20000482   Data         518  f_inobus.o(.bss)
    UartRecvBuf                              0x20000688   Data         520  f_inobus.o(.bss)
    RxDmaData                                0x20000890   Data         512  f_uart.o(.bss)
    TestBB                                   0x20000a90   Data          20  f_can_app.o(.bss)
    CanFilterTable                           0x20000aa4   Data          32  f_can_app.o(.bss)
    gCanTxBuf                                0x20000ac4   Data         164  f_can_drive.o(.bss)
    gCANRxBuf                                0x20000b68   Data         168  f_can_drive.o(.bss)
    TestAA                                   0x20000c10   Data          20  f_can_drive.o(.bss)
    ParaCode                                 0x20000c24   Data          30  f_user_main.o(.bss)
    PdoData                                  0x20000c42   Data          64  f_user_main.o(.bss)
    __initial_sp                             0x20001c88   Data           0  startup_stm32f407.o(STACK)



==============================================================================

Memory Map of the image

  Image Entry point : 0x08000189

  Load Region LR_IROM1 (Base: 0x08000000, Size: 0x00004cf8, Max: 0x00100000, ABSOLUTE)

    Execution Region ER_IROM1 (Base: 0x08000000, Size: 0x00004c54, Max: 0x00100000, ABSOLUTE)

    Base Addr    Size         Type   Attr      Idx    E Section Name        Object

    0x08000000   0x00000188   Data   RO            3    RESET               startup_stm32f407.o
    0x08000188   0x00000000   Code   RO          835  * .ARM.Collect$$$$00000000  mc_w.l(entry.o)
    0x08000188   0x00000004   Code   RO          844    .ARM.Collect$$$$00000001  mc_w.l(entry2.o)
    0x0800018c   0x00000004   Code   RO          847    .ARM.Collect$$$$00000004  mc_w.l(entry5.o)
    0x08000190   0x00000000   Code   RO          849    .ARM.Collect$$$$00000008  mc_w.l(entry7b.o)
    0x08000190   0x00000000   Code   RO          851    .ARM.Collect$$$$0000000A  mc_w.l(entry8b.o)
    0x08000190   0x00000008   Code   RO          852    .ARM.Collect$$$$0000000B  mc_w.l(entry9a.o)
    0x08000198   0x00000000   Code   RO          854    .ARM.Collect$$$$0000000D  mc_w.l(entry10a.o)
    0x08000198   0x00000000   Code   RO          856    .ARM.Collect$$$$0000000F  mc_w.l(entry11a.o)
    0x08000198   0x00000004   Code   RO          845    .ARM.Collect$$$$00002712  mc_w.l(entry2.o)
    0x0800019c   0x00000024   Code   RO            4    .text               startup_stm32f407.o
    0x080001c0   0x000000e4   Code   RO          139    .text               misc.o
    0x080002a4   0x000009ec   Code   RO          163    .text               stm32f4xx_can.o
    0x08000c90   0x00000064   Code   RO          183    .text               stm32f4xx_dbgmcu.o
    0x08000cf4   0x000003a4   Code   RO          203    .text               stm32f4xx_dma.o
    0x08001098   0x0000025c   Code   RO          263    .text               stm32f4xx_gpio.o
    0x080012f4   0x00000588   Code   RO          303    .text               stm32f4xx_rcc.o
    0x0800187c   0x00000ca2   Code   RO          345    .text               stm32f4xx_tim.o
    0x0800251e   0x00000002   PAD
    0x08002520   0x0000041a   Code   RO          365    .text               stm32f4xx_usart.o
    0x0800293a   0x00000002   PAD
    0x0800293c   0x00000120   Code   RO          405    .text               f_led.o
    0x08002a5c   0x00000448   Code   RO          536    .text               f_main.o
    0x08002ea4   0x00000220   Code   RO          583    .text               f_rcc.o
    0x080030c4   0x000002d8   Code   RO          603    .text               f_tech_comm_interface.o
    0x0800339c   0x00000088   Code   RO          631    .text               f_wwdg.o
    0x08003424   0x000000bc   Code   RO          648    .text               main.o
    0x080034e0   0x000006d8   Code   RO          673    .text               f_inobus.o
    0x08003bb8   0x000001d4   Code   RO          704    .text               f_inobusif.o
    0x08003d8c   0x00000304   Code   RO          725    .text               f_uart.o
    0x08004090   0x00000230   Code   RO          749    .text               f_can_app.o
    0x080042c0   0x000007f0   Code   RO          788    .text               f_can_drive.o
    0x08004ab0   0x00000074   Code   RO          815    .text               f_user_main.o
    0x08004b24   0x00000024   Code   RO          838    .text               mc_w.l(memcpya.o)
    0x08004b48   0x00000024   Code   RO          840    .text               mc_w.l(memseta.o)
    0x08004b6c   0x00000024   Code   RO          858    .text               mc_w.l(init.o)
    0x08004b90   0x0000000e   Code   RO          862    i.__scatterload_copy  mc_w.l(handlers.o)
    0x08004b9e   0x00000002   Code   RO          863    i.__scatterload_null  mc_w.l(handlers.o)
    0x08004ba0   0x0000000e   Code   RO          864    i.__scatterload_zeroinit  mc_w.l(handlers.o)
    0x08004bae   0x00000002   PAD
    0x08004bb0   0x00000038   Data   RO          406    .constdata          f_led.o
    0x08004be8   0x00000020   Data   RO          751    .constdata          f_can_app.o
    0x08004c08   0x0000002a   Data   RO          790    .constdata          f_can_drive.o
    0x08004c32   0x00000002   PAD
    0x08004c34   0x00000020   Data   RO          860    Region$$Table       anon$$obj.o


    Execution Region RW_IRAM1 (Base: 0x20000000, Size: 0x00001c88, Max: 0x00020000, ABSOLUTE)

    Base Addr    Size         Type   Attr      Idx    E Section Name        Object

    0x20000000   0x00000010   Data   RW          304    .data               stm32f4xx_rcc.o
    0x20000010   0x00000024   Data   RW          407    .data               f_led.o
    0x20000034   0x00000008   Data   RW          538    .data               f_main.o
    0x2000003c   0x00000014   Data   RW          605    .data               f_tech_comm_interface.o
    0x20000050   0x00000004   Data   RW          632    .data               f_wwdg.o
    0x20000054   0x00000002   Data   RW          649    .data               main.o
    0x20000056   0x00000002   PAD
    0x20000058   0x00000020   Data   RW          675    .data               f_inobus.o
    0x20000078   0x0000000b   Data   RW          705    .data               f_inobusif.o
    0x20000083   0x00000001   PAD
    0x20000084   0x00000008   Data   RW          727    .data               f_uart.o
    0x2000008c   0x00000010   Data   RW          752    .data               f_can_app.o
    0x2000009c   0x00000004   Data   RW          791    .data               f_can_drive.o
    0x200000a0   0x00000004   Data   RW          817    .data               f_user_main.o
    0x200000a4   0x00000076   Zero   RW          537    .bss                f_main.o
    0x2000011a   0x0000005e   Zero   RW          604    .bss                f_tech_comm_interface.o
    0x20000178   0x00000718   Zero   RW          674    .bss                f_inobus.o
    0x20000890   0x00000200   Zero   RW          726    .bss                f_uart.o
    0x20000a90   0x00000034   Zero   RW          750    .bss                f_can_app.o
    0x20000ac4   0x00000160   Zero   RW          789    .bss                f_can_drive.o
    0x20000c24   0x0000005e   Zero   RW          816    .bss                f_user_main.o
    0x20000c82   0x00000006   PAD
    0x20000c88   0x00001000   Zero   RW            1    STACK               startup_stm32f407.o


==============================================================================

Image component sizes


      Code (inc. data)   RO Data    RW Data    ZI Data      Debug   Object Name

       560         42         32         16         52       5814   f_can_app.o
      2032         90         42          4        352      30383   f_can_drive.o
      1752        114          0         32       1816       9073   f_inobus.o
       468         30          0         11          0       2819   f_inobusif.o
       288         12         56         36          0     260056   f_led.o
      1096         46          0          8        118       6543   f_main.o
       544         24          0          0          0       1326   f_rcc.o
       728         48          0         20         94       3593   f_tech_comm_interface.o
       772         40          0          8        512       2783   f_uart.o
       116         18          0          4         94       1856   f_user_main.o
       136          6          0          4          0       1082   f_wwdg.o
       188         12          0          2          0        746   main.o
       228         22          0          0          0       1829   misc.o
        36          8        392          0       4096        840   startup_stm32f407.o
      2540         38          0          0          0       7980   stm32f4xx_can.o
       100          4          0          0          0       1332   stm32f4xx_dbgmcu.o
       932         32          0          0          0       6305   stm32f4xx_dma.o
       604         36          0          0          0       4077   stm32f4xx_gpio.o
      1416         48          0         16          0      10943   stm32f4xx_rcc.o
      3234         60          0          0          0      22312   stm32f4xx_tim.o
      1050         26          0          0          0       7784   stm32f4xx_usart.o
         0          0          0          0          0     282192   system_stm32f4xx.o

    ----------------------------------------------------------------------
     18824        756        556        164       7140     671668   Object Totals
         0          0         32          0          0          0   (incl. Generated)
         4          0          2          3          6          0   (incl. Padding)

    ----------------------------------------------------------------------

      Code (inc. data)   RO Data    RW Data    ZI Data      Debug   Library Member Name

         0          0          0          0          0          0   entry.o
         0          0          0          0          0          0   entry10a.o
         0          0          0          0          0          0   entry11a.o
         8          4          0          0          0          0   entry2.o
         4          0          0          0          0          0   entry5.o
         0          0          0          0          0          0   entry7b.o
         0          0          0          0          0          0   entry8b.o
         8          4          0          0          0          0   entry9a.o
        30          0          0          0          0          0   handlers.o
        36          8          0          0          0         68   init.o
        36          0          0          0          0         68   memcpya.o
        36          0          0          0          0        108   memseta.o

    ----------------------------------------------------------------------
       160         16          0          0          0        244   Library Totals
         2          0          0          0          0          0   (incl. Padding)

    ----------------------------------------------------------------------

      Code (inc. data)   RO Data    RW Data    ZI Data      Debug   Library Name

       158         16          0          0          0        244   mc_w.l

    ----------------------------------------------------------------------
       160         16          0          0          0        244   Library Totals

    ----------------------------------------------------------------------

==============================================================================


      Code (inc. data)   RO Data    RW Data    ZI Data      Debug   

     18984        772        556        164       7140     668480   Grand Totals
     18984        772        556        164       7140     668480   ELF Image Totals
     18984        772        556        164          0          0   ROM Totals

==============================================================================

    Total RO  Size (Code + RO Data)                19540 (  19.08kB)
    Total RW  Size (RW Data + ZI Data)              7304 (   7.13kB)
    Total ROM Size (Code + RO Data + RW Data)      19704 (  19.24kB)

==============================================================================

